:030000000235AD19
:0C35AD0078FFE4F6D8FD75815C0235F46F
:1018610020000A3C2E2E2E3E004950436F6E6E65BD
:1018710063745245510A004950436F6E6E6563743B
:10188100000A49504E6F41434B210A003E432C56FA
:101891002C43432CC0E4E0EFF2E5F020D1E8EDEA7F
:1018A100EEEC49500A003E432C4D41432C25303289
:1018B10062583A25303262583A25303262583A2518
:1018C100303262583A25303262583A253032625805
:1018D1002C4D414320E0E4F0E5F10A003E432C5653
:1018E10045522C20332E3220EEF220257320257311
:1018F1002CC2E5F0F1E8FF20495020ECEEE4F3EBD7
:10190100FF0A004170722031382032303038003106
:10191100303A35393A3439003E432C4C442C50523C
:101921004F473A2020202020202020202020202046
:1019310020202020202020202020202020202020A6
:101941002020202020202020202020202020202096
:101951002020202020202020202020202020202086
:1019610020202020202020202CC4E0F2E020EFF0D5
:10197100EEF8E8E2EAE828F4E0E9EB290A003E2A79
:101981002C312CCEF1EDEEE2EDFBE520EFE0F0E0C5
:10199100ECE5F2F0FB20F1E5F2E5E2EEE3EE20E822
:1019A100EDF2E5F0F4E5E9F1E00A003E412C4130C9
:1019B100312C2562752E2562752E2562752E2562C4
:1019C100752C495020E0E4F0E5F120E0E4E0EFF28D
:1019D100E5F0E00A003E412C4130322C2562752EA3
:1019E1002562752E2562752E2562752C495020E0E1
:1019F100E4F0E5F120EEF1ED2E20F1E5F0E2E5F085
:101A0100E00A003E412C4130332C2562752E2562BF
:101A1100752E2562752E2562752C495020E0E4F063
:101A2100E5F120F0E5E72E20F1E5F0E2E5F0E00A4E
:101A3100003E412C4130342C2562752E2562752ED5
:101A41002562752E2562752CCCE0F1EAE020F1E5E6
:101A5100F2E80A003E412C4130352C2562752E25D5
:101A610062752E2562752E2562752CD8EBFEE70A6C
:101A7100003E2A2C312CC4EEEF2E20EFE0F0E0ECFA
:101A8100E5F2F0FB20F1E5F2E5E2EEE3EE20E8ED30
:101A9100F2E5F0F4E5E9F1E00A003E422C53303181
:101AA1002C2562752CC6E4E0F2FC20E7E0EFF0EEB5
:101AB100F1E020F1EEE5E4E8EDE5EDE8FF20EEF2FE
:101AC10020F1E5F0E2E5F0E00A003E422C5330322D
:101AD1002C2562752CCEE1ECE5ED20F120F1E5F04D
:101AE100E2E5F0EEEC20E1E5E720EAE2E8F2E0ED04
:101AF100F6E8E90A003E422C5330332C2562752C5E
:101B0100CFE5F0E5E7E0EFF3F1EA20EFF0E820EFD1
:101B1100EEF2E5F0E520F1E2FFE7E820F120F1E562
:101B2100F0E2E5F0EEEC0A003E454E440A000A44BC
:101B3100756D705820202020203030203031203029
:101B410032203033203034203035203036203037C9
:101B5100203038203039203041203042203043209D
:101B61003044203045203046000A3A003A20000A2D
:101B7100000A44756D704420202020203030203030
:101B8100312030322030332030342030352030368F
:101B91002030372030382030392030412030422069
:101BA10030432030442030452030460045727220B9
:101BB1006B657900526420656570726F6D0A005221
:101BC10064204D454D0A00526420436F64650A004C
:101BD100577269746520436F64650A0044656275D4
:101BE100674950204F4E0A0044656275674950208D
:101BF1004F46460A00446562756755736572204F0A
:101C01006E0A00446562756755736572204F4646DA
:101C11000A0044656275674D7367204F6E0A004480
:101C2100656275674D7367204F46460A00436F6EC4
:101C3100666967206C6F636B210A005772206565C6
:101C410070726F6D0A002053617665206565707250
:101C51006F6D210A00457272204D414321004C6F86
:101C610061643E3E002A003C4130313D003C413040
:101C7100323D003C4130333D003C4130343D003C7D
:101C81004130353D003C21003C5330313D003C5357
:101C910030323D003C5330333D003C5330353D0044
:061CA1003C5330363D000B
:063FAD00010B00010900F8
:103FE300C28E438910758BFF758DB7D2ABD28E22EB
:03001B0002348F1D
:10348F00C0E0C083C082C0D0C28E758BFF758DB770
:10349F0020060675A61E75A6E10509D202E50B608A
:1034AF0002050BE50AD394014002150A050EE50E3D
:1034BF00540F7048D20EE50E543F7012D200906632
:1034CF008BE0600A04F0E0D394B44002D206906619
:1034DF0086E0600204F0906104E0600214F09066F0
:1034EF008CE0D394014003E014F0300502050CE5A5
:1034FF000DD394644004D2068002050DE508D394E1
:10350F000140021508D28ED0D0D082D083D0E032C5
:10085300C2AFC291C290D2B5C20B7D027C007F07AA
:10086300123F908F24E524646060097D017F60124C
:100873003F2BD20BE4FDFC7F0B123F908F24E5242A
:1008830030E6097D04E4FF123F4FD20B7D017C006B
:100893007F07123F908F24E5247008FD7FFF123FEE
:1008A3002BD20B300B03126000C288C2A8C2AA75F8
:1008B30089001238D590633EE0B4FA06A3E064CE13
:1008C300607BE4F52474362524F582E43463F583F0
:1008D300E4F00524E524B443EC90633E74FAF0A3FA
:1008E30074CEF0A374CCF0906344740AF0E4A3F0E4
:1008F300A304F0A3F090633A74FFF0A3F0A3F0E431
:10090300A3F0906355740AF0E4F524E5242401FF71
:10091300E433FE74362524F582E43463F583E0FD85
:10092300123F070524E524C3944340DFE4F5A7758C
:10093300A61E75A6E1907FF0F0A3F080FE906349B8
:100943007403F0A374CCF0E4906348F0123315C23F
:10095300B5123A47C206123D91D20BC20DC20C909A
:1009630065767408F09062B47424F0E4A3F09063A5
:100973003EE09062B6F090633FE09062B7F0906320
:1009830040E09062B8F0906341E09062B9F0906308
:1009930042E09062BAF0906343E09062BBF0750A64
:1009A30001E4906577F0C207C208C209C20A200BAE
:1009B30018AF24FE7D03123158E4FF1233DF7E1893
:1009C3007F61E4FBFDFC122D7590668BE060037480
:1009D30001F0E4906104F0F50C906575F0F50D12EB
:1009E3003FE375A70775A61E75A6E1D2AFE4F50D23
:1009F300906104E07003120EB190668CE0B40111B3
:100A03009080007410F0E490668CF0D20BC20CC29C
:100A13000D908008E0F52430E405D2077410F0E56A
:100A23002430E508D2099080087420F0E52430E6EC
:100A330008D2089080087440F0E50CC39403401971
:100A4300908002E4F0908001F0908000F0E50C9437
:100A5300064006E4F50C123D919080A0E07003126D
:100A630039539080B8E070031239CD9080D0E07094
:100A730003123C0E908000E07013300710122E7C9E
:100A8300906331EFF0D3940040031200269080026C
:100A9300E07006908000E06005D2050209F0C2050F
:100AA300E4F50C906104E060030209F0200B12905E
:100AB3006578E0600C7E187F63123070E49065788F
:100AC300F03009121229F2906331EFF0D394004011
:100AD30005E0FF123FF7200803020C5912286B9020
:100AE3006331EFF070030209F0906375E054BF24A3
:100AF3007F7003020BC2147003020B9A240260037B
:100B0300020BFB200B077E187F6A123070200F0345
:100B1300020C5990634DE07006906351E06067905A
:100B23006682E0FF90634DE0B50724906683E0FEA4
:100B330090634EE0B50618906684E0FE90634FE044
:100B4300B5060C906685E0FE906350E06E603790CA
:100B53006351E06F6003020C59906683E0FF90637A
:100B630052E06F6003020C59906684E0FF90635378
:100B7300E06F6003020C59906685E0FF906354E0D8
:100B83006F6003020C59C2039065777401F0123F42
:100B9300FA750A01020C5990668BE060037401F048
:100BA30090667AE0FF906377E06F6003020C5990E0
:100BB300667AE004F0E4F50A906575F0020C5930AA
:100BC3000303020C59906344E070030209F090633D
:100BD30055740AF012001ED203E4F50A906575F00D
:100BE30090668604F0E4906679F0A3F0200B677EAC
:100BF300187F78123070805E90668BE0600374011A
:100C0300F0300352906375E020E74B906377E0FF89
:100C1300906679E0FE6F600D906681E07007EE14D8
:100C23006F70338013906679E004F0906331E0FFD6
:100C3300D394044003123FF99060007482F0A374CC
:100C430001F0906377E0906002F07E607F007D03A7
:100C53001236C00209F0200303020D71E50A706821
:100C630012351FEF60237E647F75906476E0240461
:100C7300FD1236C0906681E07009906355E0F50A75
:100C83000209F0E4F50A0209F0906686E0D3943C89
:100C93004036906681E0703090668604F0123FF82B
:100CA300E4906475F0A37412F090667AE090647730
:100CB300F0A374FDF090610563A20190647963A2CF
:100CC300017F121225B9809E123FF38F24E524B4CD
:100CD30001159060007483F0E4A3F07E607F007DD3
:100CE300021236C00209F0E524D39401401C90603F
:100CF300007483F0A37401F0E52424FEA3F07E6066
:100D03007F007D031236C00209F0E50A6401600327
:100D13000209F0906575E004F0200B077E187F82CE
:100D2300123070906355E0C394C85004E02432F04D
:100D3300906575E0C39405400DC203E4906577F0B8
:100D4300123FFA0209F07C667D82906349E0FAA3C0
:100D5300E0FB7F021238517E647F75906476E02455
:100D630004FD1236C0906355E0F50A0209F0E50A66
:100D7300640160030209F0906577E014604624FE85
:100D83006042147003020E64240460030209F0E459
:100D9300F50C200F139065777404F0906575E0549B
:100DA30001F0750A010209F09080027410F0E490DA
:100DB3006577F090657504F0750AFA90668274FFA2
:100DC300F00209F0906682E07003020E4E906475A3
:100DD3007480F09064777401F0E4A3F0A304F0A3AB
:100DE3007430F0A3747BF0E4F524747C2524F5823D
:100DF300E43464F583747DF0747D2524F582E43452
:100E030064F583E4F0E5242407906476F07C667D42
:100E130082906349E0FAA3E0FB7F021238517E64BB
:100E23007F75E5242409FD1236C0906681E0601BBE
:100E330012001ED203E4F50A906575F090668604ED
:100E4300F0E4906679F0A3F00209F0300F07E49024
:100E53006577F080069065777404F0750AFA0209E5
:100E6300F09080027410F0750A05906575E06401D6
:100E7300FFF09065777401F0EF7019906351E060B3
:100E830013FCA3E0FDA3E0FEA3E0FF906682122122
:100E9300940209F090634DE0FCA3E0FDA3E0FEA300
:0D0EA300E0FF9066821221940209F080FEAB
:010EB000221F
:10002600906376E0B444047F0180027F009063759C
:10003600E0B447047E0180027E00EE5F604A906372
:100046003EE0906377F090633FE0906378F09063D2
:1000560040E0906379F0906341E090637AF09063BA
:1000660042E090637BF0906343E090637CF09063A2
:10007600767452F09062AE63A2019080A863A201EA
:100086007F061225B9020849906331E0C3940850EF
:100096000302085290633EE0FF906377E06F6003CF
:1000A60002085290633FE0FF906378E06F600302BE
:1000B6000852906340E0FF906379E06F60030208A6
:1000C60052906341E0FF90637AE06F60030208524A
:1000D600906342E0FF90637BE06F600302085290FA
:1000E6006343E0FF90637CE06F6003020852906315
:1000F60076E0B444159062AEE0B4FF0E63A20190C0
:1001060080A863A2017F061225B990668BE0600382
:100116007401F090668C7464F09063767452F0907B
:100126006375E0646D60030202537BFF7A18798D74
:10013600121D097BFF7A1879A790633EE0F52EA37E
:10014600E0F52FA3E0F530A3E0F531A3E0F532A307
:10015600E0F533121D09752EFF752F1975300475DC
:1001660031FF7532197533107BFF7A1879DD121D50
:10017600097BFF7A197919121D097BFF7A19797F94
:10018600121D097BFF7A1979AC906344E0F52EA322
:10019600E0F52FA3E0F530A3E0F531121D097BFF52
:1001A6007A1979D690634DE0F52EA3E0F52FA3E0FA
:1001B600F530A3E0F531121D097BFF7A1A79049018
:1001C6006351E0F52EA3E0F52FA3E0F530A3E0F5AB
:1001D60031121D097BFF7A1A793290633AE0F52EC7
:1001E600A3E0F52FA3E0F530A3E0F531121D097B5E
:1001F600FF7A1A7955906336E0F52EA3E0F52FA322
:10020600E0F530A3E0F531121D097BFF7A1A797209
:10021600121D097BFF7A1A799BA20FE433F52E1281
:100226001D097BFF7A1A79CB906681E0F52E121DA7
:10023600097BFF7A1A79F690668BE0F52E121D0976
:10024600122B587BFF7A1B7929121D0922906375A0
:10025600E0644C70737E1B7F2FFBFDFC122D7590A6
:10026600637DE0F525A3E0F526E4F528E525906312
:100276007FF0A3E526F07E1B7F6A7C637D7F7B0291
:10028600122D75E4F527852682852583E0FF747F88
:100296002527F582E43463F583EFF00526E526701D
:1002A6000205250527E527B410DC7E1B7F6D7C63E0
:1002B6007D7F7B10122D750528E528C3941040AC70
:1002C6007E1B7F7012307022906375E0646C7060E4
:1002D600F5297E1B7F72FBFDFC122D75E4F528E4E3
:1002E60090637FF0A3E529F07E1B7F6A7C637D7FA8
:1002F6007B02122D75E4F527A829E6FF747F2527D2
:10030600F582E43463F583EFF005290527E527B484
:1003160010E67E1B7F6D7C637D7F7B10122D75053D
:1003260028E528C3940840B77E1B7F7012307022E0
:10033600906375E0644B7061F52774672527F58235
:10034600E43463F583E0603274672527F582E4348C
:1003560063F583E0F4602374672527F582E434634C
:10036600F583E0FF747D2527F582E43463F583E0A9
:10037600B507100527E527B408C09061047432F06C
:100386000208499063757421F0300B030208497E18
:100396001B7FAD123070020849906375E0B4521AA3
:1003A600200B077E1B7FB51230709063757472F058
:1003B6007E637F757D0812363922906375E0644945
:1003C6007045200B077E1B7FC012307090637DE066
:1003D600F525A3E0F526E4F527852682852583E025
:1003E600FF747F2527F582E43463F583EFF0052655
:1003F600E526700205250527E527B480DC7E637FA8
:10040600757D8A12363922906375E0644370462002
:100416000B077E1B7FC812307090637DE0F525A325
:10042600E0F526E4F527852682852583E493FF7487
:100436007F2527F582E43463F583EFF00526E5266C
:10044600700205250527E527B480DB7E637F757D71
:100456008A12363922906375E0645A7053200B076E
:100466007E1B7FD112307090637DE0F525A3E0F509
:10047600267C637D7F7B80AF26AE25123EADE4F5FC
:1004860027852682852583E493FF747F2527F582B9
:10049600E43463F583EFF00526E5267002052505AD
:1004A60027E527B480DB7E637F757D8A1236392285
:1004B600906375E06444600302054790637DE0FF46
:1004C60064447003020849EFB4310CC20B7E1B7FF3
:1004D600DD12307002084990637DE0B4300CD20B17
:1004E6007E1B7FE912307002084990637DE0B432CA
:1004F6000CD20C7E1B7FF612307002084990637D89
:10050600E0B4330CC20C7E1C7F0412307002084922
:1005160090637DE0B4340CD20D7E1C7F13123070D4
:1005260002084990637DE0B4350CC20D7E1C7F2025
:1005360012307002084990637DE0FF123FF6020810
:1005460049906104E07013200B077E1C7F2E123049
:10055600709063757421F00208499061047432F05A
:10056600906375E0FFB45104C2AF80FEEF6457702C
:1005760045200B077E1C7F3C12307090637EE09016
:100586006331F0E4F527906331E0FFE527C39F4030
:1005960003020849747F2527F582E43463F583E076
:1005A600FF90637DE0252724ADF582E43461F58371
:1005B600EFF0052780D0906375E064536003020670
:1005C6006A200B077E1C7F4712307090633EE0FF67
:1005D6009061B6E06F703C90633FE0FF9061B7E0DA
:1005E6006F7030906340E0FF9061B8E0B5072490EB
:1005F6006341E0FF9061B9E0B50718906342E0FF00
:100606009061BAE0B5070C906343E0FF9061BBE0F0
:100616006F60169063757421F0300B030208497EF3
:100626001C7F56123070020849E4F527E4F50DAF39
:1006360027FE74AD2527F582E43461F583E0FD12CB
:100646003F070527E527C394FE40E1C2AFE4907F4C
:10065600F0F0A3F0907FFD74AAF0A374FFF0A374EA
:1006660055F080FE906375E0644F704C90637DE0BA
:10067600F525A3E0F526E5264525700A200B077E1D
:100686001C7F5F123070200B077E1C7F6612307055
:10069600E4F527747F2527F582E43463F583E08546
:1006A6002682852583F00526E52670020525052781
:1006B600E527B480DE020849906375E0FFB4452162
:1006C60090637DE0FDA3E0907FF0CDF0A3EDF0C256
:1006D600AF907FFD74AAF0A374FFF0A37455F08069
:1006E600FEEF6465600302085290637DE0FFA3E0BD
:1006F600907FF0CFF0A3EFF0E4F525F526D3907FB9
:10070600F1E09526907FF0E095254020E4F50D2553
:1007160026FFE5253401FE852682852583E0FD1228
:100726003F070526E5267002052580D17E1C7F68D9
:10073600123747EF4E6020120003906344EFF01229
:100746000003906345EFF0120003906346EFF0124A
:100756000003906347EFF07E1C7F6E123747EF4E23
:10076600602012000390634DEFF012000390634E79
:10077600EFF012000390634FEFF012000390635006
:10078600EFF07E1C7F74123747EF4E602012000395
:10079600906351EFF0120003906352EFF0120003E2
:1007A600906353EFF0120003906354EFF07E1C7FCA
:1007B6007A123747EF4E602012000390633AEFF04B
:1007C60012000390633BEFF012000390633CEFF0DE
:1007D60012000390633DEFF07E1C7F80123747EFD7
:1007E6004E6020120003906336EFF0120003906310
:1007F60037EFF0120003906338EFF01200039063B6
:1008060039EFF0E4F527E4F50DE5272401FFE4339D
:10081600FE74362527F582E43463F583E0FD123F46
:10082600070527E527C3944340DCC2AFE4907FF079
:10083600F0A3F0907FFD74AAF0A374FFF0A37455A3
:0C084600F080FE7E637F757D081236395D
:010852002283
:103E7500AE07EEC39430400BEED394395005EE24D3
:103E8500D0FF22EEC39461400BEED394665005EE4D
:103E950024A9FF22EEC39441400BEED3944650056E
:083EA500EE24C9FF22AF062242
:103FC9009062ADE004F070069062ACE004F090629B
:0A3FD900ACE0FEA3E0FF123F7322EC
:10000300123FC9123E75EFC454F0FEC006123FC939
:08001300123E75D0E02FFF2220
:103D3400E4906B8AF0123FC9906B8BEFF0C3943020
:103D44004018E0FFD394395011906B8AE02405F5B4
:103D540082E43461F583EFF08011906B8AE02405EE
:103D6400F582E43461F583E4F0800C906B8AE0041E
:103D7400F0E0D3940840BE752D00752E00752F0019
:0C3D8400E4F5307B017A6179051226C756
:013D90002210
:043747008E2A8F2B0C
:10374B009062ACE4F0A374FFF0123FC9EF606EF42B
:10375B00606B852B82852A83E493B507EC752C016E
:10376B00E52B252CF582E4352AF583E4936025902F
:10377B0062ADE0252CFF9062ACE03400FE123F738B
:10378B00E52B252CF582E4352AF583E493B5070464
:10379B00052C80CCE52B252CF582E4352AF583E42A
:1037AB009370A6E52C24FFFFE434FFFE9062ADE09E
:1037BB002FF09062ACE03EF07E007F0122E4FEFF32
:0137CB0022DB
:103315007E1C7F86123747EF4E70037F01227E1C8D
:103325007F89123747EF4E600C123FC9EF24D02436
:10333500FF920F8002D20F7E1C7F8F123747EF4E10
:10334500600C123FC9EF24D0906681F08005E490AF
:103355006681F07E1C7F95123747EF4E600C123F59
:10336500C9EF24D090668BF08005E490668BF07EE3
:103375001C7F9B123747EF4E600C123FC9EF24D0DC
:1033850024FF92018002C20190633E63A201906610
:103395007B63A2017F061225B930013B7E1C7FA10C
:1033A500123747EF4E603012000390667BEFF01244
:1033B500000390667CEFF012000390667DEFF0123B
:1033C500000390667EEFF012000390667FEFF01227
:0A33D5000003906680EFF07F0022F5
:103DEA00906576E0C3947C503D906576E0FE04F0E1
:103DFA0074B42EF582E43462F583EFF0BF0A27909B
:103E0A006576E0FF04F074B42FF582E43462F5833A
:103E1A00E4F0906576E0FF1237CC9065767408F08E
:073E2A009062B5E004F022F4
:103D91009080007480F090633663A201F583F58210
:103DA10063A2017F081225B990633E63A20190804E
:103DB1008863A2017F0A1225B9908092E4F0A3746E
:103DC10032F0A37401F0906348E0FF9080B1F0906D
:103DD10080E1EFF09080957455F0A3F0908000742D
:093DE10001F090800974F0F02259
:10395300908009E04410F09080A0E0706C9080A10A
:103963007482F09080A874FFF0A3F0A3F0A3F07F1B
:10397300039080AEEFF07FCBA3EFF07F039080AC9A
:10398300EFF0A374CBF09080007402F0906B7E1282
:1039930021A000000000906B7EE0908040F0906BCF
:1039A3007FE0908041F0906B80E0908042F0906BDC
:1039B30081E0908043F0A3E4F0A3F0A3F0A3F090A0
:0939C3008018F0A3F0A3F0A3F0BA
:0139CC0022D8
:103C0E00908009E04440F09080D17482F090634936
:103C1E00E0FF9080DEF090634AE0FF9080DFF0904E
:103C2E0080027402F0906B821221A00000000090BE
:103C3E006B82E0908058F0906B83E0908059F0900A
:103C4E006B84E090805AF0906B85E090805BF0A3DF
:103C5E00E4F0A3F0A3F0A3F0908030F0A3F0A3F073
:023C6E00A3F0C1
:013C70002231
:1039CD00908009E04420F09080B8E0706C9080B950
:1039DD007482F07F039080C6EFF07FCDA3EFF07F70
:1039ED00039080C4EFF0A374CDF09080C074FFF00D
:1039FD00A3F0A3F0A3F09080017402F0906B8612F7
:103A0D0021A000000000906B86E090804CF0906B40
:103A1D0087E090804DF0906B88E090804EF0906B39
:103A2D0089E090804FF0A3E4F0A3F0A3F0A3F09011
:093A3D008024F0A3F0A3F0A3F033
:013A4600225D
:103851008C258D26A907EAFDE975F018A424ACFF93
:10386100E5F034808F82F583EDF0EBFDE975F0181A
:10387100A4FFAEF024ACFBEE34808B82F583A3ED84
:10388100F08526828C83E0FDEF24A8FFEE3480FED4
:103891008F82F583EDF08526828C83A3E08F828E63
:1038A10083A3F0852682852583A3A3E0FDE975F036
:1038B10018A424A8FFE5F03480FE8F82F583A3A32A
:1038C100EDF08526828C83A3A3A3E08F828E83A350
:0438D100A3A3F0229B
:063639008D2AAB07AA0672
:10363F00908000E030E5079065787401F022906B80
:10364F007EE0FCA3E0FDA3E0FEA3E0F52E8E2D8D22
:10365F002C8C2BAE02AF038E838F8263A201E52DDC
:10366F00540744C0F583852E8263A201AF2A122628
:10367F002BE4FCFDFEE52E252AF52EEE352DF52D3E
:10368F00ED352CF52CEC352BF52B908040E52BF000
:10369F00A3E52CF0A3E52DF0A3E52EF090800074A8
:1036AF0020F0AF2EAE2DAD2CAC2B906B7E12219453
:0136BF0022E8
:0636C0008D25AB07AA06F0
:1036C600908002E030E5079065787403F022906BF5
:1036D60082E0FCA3E0FDA3E0FEA3E0F5298E288DA1
:1036E600278C26AE02AF038E838F8263A201E52864
:1036F600540744D0F58385298263A201AF2512269B
:103706002BE4FCFDFEE5292525F529EE3528F528CF
:10371600ED3527F527EC3526F526908058E526F079
:10372600A3E527F0A3E528F0A3E529F0908002742D
:1037360020F0AF29AE28AD27AC26906B82122194DB
:013746002260
:0233DF008F2538
:1033E100908001E030E5099065787402F07F002259
:1033F100906B86E0FCA3E0FDA3E0FEA3E0F5298E3F
:10340100288D278C2690667B63A201E5285407440A
:10341100C8F58385298263A2017F06122641E52929
:103421002406F529E43528F528E43527F527E43580
:1034310026F52690657963A201E528540744C8F56D
:103441008385298263A201AF25122641E4FCFDFE9A
:10345100E5292525F529EE3528F528ED3527F52728
:10346100EC3526F52690804CE526F0A3E527F0A360
:10347100E528F0A3E529F09080017420F0AF29AE92
:0D34810028AD27AC26906B86122194AF2554
:01348E00221B
:102E7C009081E0E0F5250525052505250525052589
:102E8C0005250525052505250525908010E0F52847
:102E9C00A3E0F529A3E0F52AA3E0F52B9081E1E06E
:102EAC00F5250525052505250525052505250525D6
:102EBC00052505250525908014E0F52CA3E0F52DBE
:102ECC00A3E0F52EA3E0F52FE52EB52A08E52FB5E6
:102EDC002B037F0022E4F525E52E540744E0F5830F
:102EEC00852F8263A20190637563A2017F0812266D
:102EFC007190637763A2019062AE63A2017F0612A8
:102F0C0025B9906375E0F526A3E0F527E4F5259047
:102F1C006375E0702AA3E024F8F525E52E540744E8
:102F2C00E0F583852F8274082582F582E43583F5DC
:102F3C008363A20190637563A201AF25122671AE63
:102F4C0026E4FCFDE52F2527F52FE52E3EF52EED8D
:102F5C00352DF52DEC352CF52C908014E52CF0A3AB
:102F6C00E52DF0A3E52EF0A3E52FF0908000744042
:032F7C00F0AF258E
:012F7F00222F
:10286B009081E6E0F525052505250525052505259A
:10287B0005250525052505250525908028E0F52846
:10288B00A3E0F529A3E0F52AA3E0F52B9081E7E07F
:10289B00F5250525052505250525052505250525ED
:1028AB0005250525052590802CE0F52CA3E0F52DBD
:1028BB00A3E0F52EA3E0F52FE4F525E52EB52A0AC6
:1028CB00E52FB52B05C2080229D7E52E540744F096
:1028DB00F583852F8263A20190637563A2017F0844
:1028EB00122671906375E0F526A3E0F527E52745E1
:1028FB002670099080027410F07F0022906682E0AF
:10290B00FFF46030906377E06F600302299E90665E
:10291B0083E0FF906378E06F7079906684E0FF90BE
:10292B006379E06F706D906685E0FF90637AE06F7E
:10293B006031805F906377E0906682F0906378E01F
:10294B00906683F0906379E0906684F090637AE010
:10295B00906685F090637BE0FFA3E0906349CFF036
:10296B00A3EFF0906375E0702AA3E024F8F525E55A
:10297B002E540744F0F583852F8274082582F58247
:10298B00E43583F58363A20190637563A201AF25E0
:10299B00122671AE26E4FCFDE52F2527F52FE52E3B
:1029AB003EF52EED352DF52DEC352CF52CAF2BAE54
:1029BB002AAD29AC28AB2FAA2EA92DA82CD31221D6
:1029CB008340099080027410F07F002290802CE5E8
:1029DB002CF0A3E52DF0A3E52EF0A3E52FF09080CE
:0629EB00027440F0AF256C
:0129F10022C3
:1029F2009081E3E0F5250525052505250525052515
:102A02000525052505250525052590801CE0F528C9
:102A1200A3E0F529A3E0F52AA3E0F52B9081E4E0F9
:102A2200F525052505250525052505250525052564
:102A3200052505250525908020E0F52CA3E0F52D40
:102A4200A3E0F52EA3E0F52FE4F525E52EB52A0A3D
:102A5200E52FB52B05C209022B3DE52E540744E8AC
:102A6200F583852F8263A20190600463A2017F0E29
:102A7200122687906004E0F526A3E0F52790600C0B
:102A8200E0FFF4604590667BE0FEEF6E706EA3E0BF
:102A9200FF90600DE06F706490667DE0FF90600EC5
:102AA200E06F705890667EE0FF90600FE06F704CB0
:102AB20090667FE0FF906010E06F7040906680E06B
:102AC200FF906011E06F60048032D2D9906004E020
:102AD200702AA3E024F2F525E52E540744E8F58395
:102AE200852F82740E2582F582E43583F58363A2F5
:102AF2000190600463A201AF25122687AE26E4FC92
:102B0200FDE52F2527F52FE52E3EF52EED352DF58A
:102B12002DEC352CF52CAF2BAE2AAD29AC28AB2FE2
:102B2200AA2EA92DA82CD31221835006E5274526CB
:102B320070099080017410F07F0022908020E52CB3
:102B4200F0A3E52DF0A3E52EF0A3E52FF090800190
:052B52007440F0AF2506
:012B5700225B
:043070008E2A8F2BEA
:10307400908000E030E5079065787401F022906B51
:103084007EE0FCA3E0FDA3E0FEA3E0F5318E308DED
:103094002F8C2EE531FFE5305407FEE42FF52DEE9D
:1030A40034C0F52C852D82F5837423F0052DE52D90
:1030B4007002052C532CC7F582852C83740AF00505
:1030C4002DE52D7002052C532CC790633E63A2019D
:1030D400852C83852D8263A2017F0612262B74061C
:1030E400252DF52DE4352CF52C852A83852B82633B
:1030F400A201852C83852D8263A20112260FE4FC94
:10310400FDFE906B7EE0F8A3E0F9A3E0FAA3E02FC4
:10311400FFEE3AFEED39FDEC38FCEF2408FFE43E07
:10312400FEE43DFDE43CFC906B7E122194906B7EAA
:10313400E0908040F0906B7FE0908041F0906B8055
:10314400E0908042F0906B81E0908043F0908000AA
:033154007420F0F4
:013157002255
:0A2D75008E2A8F2B8C2C8D2D8B2EB7
:102D7F00908000E030E5079065787401F022906B49
:102D8F007EE0FCA3E0FDA3E0FEA3E0F5348E338DDF
:102D9F00328C31E534FFE5335407FEE42FF530EE86
:102DAF0034C0F52F853082F5837423F00530E5307C
:102DBF007002052F532FC7F582852F83740AF005F4
:102DCF0030E5307002052F532FC790633E63A20189
:102DDF00852F8385308263A2017F0612262B74060E
:102DEF002530F530E4352FF52F852A83852B826327
:102DFF00A201852F8385308263A20112260F8F35A2
:102E0F00EF2530F530E4352FF52FE52E6017852CA3
:102E1F0083852D8263A201852F8385308263A20172
:102E2F00AF2E12262BE5352408252EF52EFFE4FCB8
:102E3F00FDFEE5342FF534EE3533F533ED3532F550
:102E4F0032EC3531F531908040E531F0A3E532F0C9
:102E5F00A3E533F0A3E534F09080007420F0AF3495
:0C2E6F00AE33AD32AC31906B7E1221947A
:012E7B002234
:0237CC008F3F2D
:1037CE00908000E030E5079065787401F022906BF0
:1037DE007EE0FCA3E0FDA3E0FEA3E0F5438E428D68
:1037EE00418C40E543FFE5425407FEE42FFFEE34E3
:1037FE00C09062B463A201F5838F8263A201AF3FD2
:10380E0012262BE4FCFDFEE543253FF543EE354243
:10381E00F542ED3541F541EC3540F540908040E5FF
:10382E0040F0A3E541F0A3E542F0A3E543F090801C
:10383E00007420F0AF43AE42AD41AC40906B7E12AF
:02384E002194C3
:013850002255
:063158008E2A8F2BAB054F
:10315E00908000E030E5079065787401F022906B66
:10316E007EE0FCA3E0FDA3E0FEA3E0F5318E308D02
:10317E002F8C2EE531FFE5305407FEE42FF52DEEB2
:10318E0034C0F52C852D82F5837423F0052DE52DA5
:10319E007002052C532CC7F582852C83EBF0052D80
:1031AE00E52D7002052C90633E63A201852C83856C
:1031BE002D8263A2017F0612262B7406252DF52D76
:1031CE00E4352CF52C532CC7E52A852D82852C83CE
:1031DE00F0052DE52D7002052C532CC7F582852C9C
:1031EE0083E52BF0052DE52D7002052C532CC7E53C
:1031FE0031240AF531E43530F530E4352FF52FE47E
:10320E00352EF52E908040E52EF0A3E52FF0A3E5A8
:10321E0030F0A3E531F09080007420F0AF31AE3085
:0A322E00AD2FAC2E906B7E122194A0
:013238002273
:103C7100908009E04480F09080E97401F07F099020
:103C810080F6EFF0A37464F09080037402F09080EA
:103C910000E020E1F9906A7A1221A0000000009072
:103CA1006A7AE0908064F0906A7BE0908065F090A1
:103CB1006A7CE0908066F0906A7DE0908067F0A376
:103CC100E4F0A3F0A3F0A3F090803CF0A3F0A3F004
:023CD100A3F05E
:013CD30022CE
:103239009081E9E0F52805280528052805280528AD
:1032490005280528052805280528908034E0F52952
:10325900A3E0F52AA3E0F52BA3E0F52C9081EAE0A1
:10326900F5280528052805280528052805280528FD
:10327900052805280528908038E0F52DA3E0F52ECE
:10328900A3E0F52FA3E0F530E52FB52B08E530B520
:103299002C037F0022AF30AE2FAD2EAC2DAB2CAA64
:1032A9002BA92AA829D3122183400AAF30AE2CEECC
:1032B9009FF528800AAF30EFF404AE2C2EF528E5EF
:1032C9002F540744E0F58385308263A201906A7E1A
:1032D90063A201AF2812269FE4FCFDFEE5302528F4
:1032E900F530EE352FF52FED352EF52EEC352DF584
:1032F9002D908038E52DF0A3E52EF0A3E52FF0A35E
:0B330900E530F09080037440F0AF2826
:013314002296
:022F80008F2898
:102F82009080E8E0640660037FFF22906A7AE0FCAA
:102F9200A3E0FDA3E0FEA3E0F52C8E2B8D2A8C2965
:102FA200E4FFFEFDFCAB2CAA2BA92AA829C31221FF
:102FB2008370609081F9E0F529906A7AE0FCA3E0E1
:102FC200FDA3E0FEA3E0FFE4FAF9F8EF2401FFEA33
:102FD2003EFEE93DFDE83CFC906A7A122194906A3B
:102FE2007AE0FCA3E0FDA3E0FEA3E0FFE4F8EF2417
:102FF20001FFEA3EFEE93DFDE83CFC906A7A1221BF
:1030020094908064E0F529A3E0F52AA3E0F52BA3D0
:10301200E0F52C906A7E63A201E52B540744D8F5B3
:1030220083852C8263A201AF28122659E4FCFDFE9F
:10303200E52C2528F52CEE352BF52BED352AF52A36
:10304200EC3529F529908064E529F0A3E52AF0A35F
:10305200E52BF0A3E52CF09080037420F0AF2CAEAA
:0D3062002BAD2AAC29906A7A1221947F00D0
:01306F00223E
:103F7300A2AF9210C2AF438E2075D2028F828E837E
:0C3F8300E0FFE4F5D2538EDFA21092AFF5
:013F8F00220F
:103F0700E5D220E0FBA2AF9210C2AF43D2028F826C
:103F17008E83EDF075D25063D250A21092AFE5D2E6
:033F270020E0FB9C
:013F2A002274
:1038D500E4FDED2401FFE433FE123F7374362DF54C
:1038E50082E43463F583EFF00DBD3FE6E4FDED249E
:1038F5007FFFE433FE123F73742D2DF582E43461AE
:10390500F583EFF0742D2DF582E43461F583E070D5
:103915001B742D2DF582E43461F5837420F0742E2B
:103925002DF582E43461F583E4F080040DBD80BE9D
:10393500E49061ACF0FDEDFF7E00123F7374AD2D98
:0D394500F582E43461F583EFF00DBDFEE97D
:013952002252
:023EAD008B2A5E
:103EAF00A2AF9210C2AF85A22B53A2FE8E838F8238
:103EBF0005A28C838D8274091226B5E52A53A2FEC2
:103ECF0043A2201226B753A2DF852BA2A21092AFD6
:013EDF00FFE3
:013EE00022BF
:103F9000A2AF9210C2AF8C838D82EF1226B543A2DE
:0C3FA000201226B753A2DFA21092AFFF40
:013FAC0022F2
:023F2B008F25E0
:103F2D00A2AF9210C2AFE4F5838D8274061226B54E
:103F3D00E52543A2201226B753A2DFA21092AF7F30
:013F4D000172
:013F4E002250
:023F4F008F25BC
:103F5100A2AF9210C2AFE4F5838D82740A1226B526
:103F6100E52543A2201226B753A2DFA21092AF7F0C
:013F7100014E
:013F7200222C
:1024DE00A907E7FFA805EF93C3966008403B74FC7D
:1024EE002FFF80F00F08EF93C3966008402B74FB0C
:1024FE002FFF80E00F08EF93C3966008401B74FA1D
:10250E002FFF80D00F08EF93D3966008400B74F91D
:10251E002FFF80C01F1F1F1F1FEF54FEF80303F76E
:10252E00E893FC08E893FD08E893FE08E893FF2281
:10253E0009E993C39D6008402974FB29F980F109CC
:10254E00E993C39E6008401A74FA29F980E209E9FA
:10255E0093D39F6008400B74F929F980D319191988
:10256E001919E9C313C313FF22740093F8ECC3982F
:10257E004024701F740193F8EDC3984019701474C1
:0E258E000293F8EEC398400E7009740393F8A0
:10259C00EFC39840037F00227F0122EDF8E6F0089C
:1025AC00A3DFFA22EDF8E0F608A3DFFA22E0A3633A
:1025BC00A201F0A363A201DFF475A2002263A201C1
:1025CC00F0A363A20122E0A363A201F0A363A20122
:1025DC00E0A363A201F0A363A201E463A201F0A350
:1025EC0063A201DFE175A20022E0A363A2016DFEEC
:1025FC00936CFDEE058393FC158363A201DFEA75F2
:10260C00A200227F00E493A363A201F00F600CA34D
:10261C00E583C2E3F58363A20180EA75A20022E0A0
:10262C00A363A201F0A3E583C2E3F58363A201DFF8
:10263C00EE75A20022E0A363A201F0A3E583C2E43D
:10264C00D2E3F58363A201DFEC75A20022E0A36361
:10265C00A201F0A3E58344F8C2E5F58363A201DF90
:10266C00EC75A20022E583C2E3F583E0A363A2012B
:10267C00F0A363A201DFEE75A20022E583C2E4D2CF
:0A268C00E3F583E0A363A201F0A3CD
:1026960063A201DFEC75A20022E58344F8F583E02E
:1026A600A363A201F0A363A201DFEE75A20022F9E3
:1026B60022C002C004C00612FFF0D006D004D00229
:0126C60022F1
:1013F9003E2A2C312CCFE0F0E0ECE5F2F0FB20F8AE
:10140900E8EDFB2043414E0A003E4C2C6B30312C59
:1014190025732C43EAEEF0EEF1F2FC20EDE020F822
:10142900E8EDE52043414E2C30202D20353030EABF
:10143900E1283530EC292C31202D203530EAE128FE
:10144900353030EC290A0030202D20353030EAE1E2
:10145900283530EC290031202D203530EAE12835B6
:101469003030EC29003E2A2C312CCFE0F0E0ECE5BD
:10147900F2F0FB20EFF0EEF2EEEAEEEBE0204D4F5A
:10148900444255530A003E4C2C4930312C256C7589
:101499002CD1EAEEF0EEF1F2FC20EEE1ECE5EDE024
:1014A9002C343830302C393630302C313932303018
:1014B9000A003E532C4931322C2562752CC0E4F0C8
:1014C900E5F120E1EBEEEAE020D2C8D220EDE02000
:1014D900F8E8EDE50A003E532C6D2562752C25626E
:1014E900752D25752D2562752D2562752CC7E0EFA3
:1014F900F0EEF1202562752028B9CFF02DD0E5E373
:101509002DCAEEEB2DD2E8EF290A003E532C5630B6
:10151900382C25752CCFE0F3E7E020E220EEEFF040
:10152900EEF1E0F528ECF1290A003C21003C6B3092
:10153900313D003C4930313D003C4931323D003CB0
:101549005630383D002043616E45724749540020AA
:101559000A002043616E457272434821000A00491E
:101569006E69745443500A004C697374656E544330
:10157900500A00534F434B5F5443505F4553544106
:10158900424C49534845440A000A2D3E20000A3C72
:101599002D2000CEF2E2E5F23A00CEF8E8E1EAE0E9
:1015A90020CAD12100CEF8E8E1EAE020E0E4F0E544
:1015B900F1E02100CEF8E8E1EAE020F2E8EFE021ED
:1015C90000CEF8E8E1EAE020E4EBE8EDFB21000ACF
:1015D900C7E0EFF0EEF13A003C6D303D000000004D
:1015E9003C6D313D000000003C6D323D00000000C3
:1015F9003C6D333D000000003C6D343D00000000AF
:101609003C6D353D000000003C6D363D000000009A
:101619003C6D373D000000003C6D383D0000000086
:101629003C6D393D000000003C6D31303D0000004B
:101639003C6D31313D0000003C6D31323D00000010
:101649003C6D31333D0000003C6D31343D000000FC
:101659003C6D31353D00000000C1814001C0804131
:1016690001C0804100C1814001C0804100C1814069
:1016790000C1814001C0804101C0804100C1814059
:1016890000C1814001C0804100C1814001C0804149
:1016990001C0804100C1814001C0804100C1814039
:1016A90000C1814001C0804100C1814001C0804129
:1016B90001C0804100C1814000C1814001C0804119
:1016C90001C0804100C1814001C0804100C1814009
:1016D90000C1814001C0804101C0804100C18140F9
:1016E90000C1814001C0804100C1814001C08041E9
:1016F90001C0804100C1814000C1814001C08041D9
:1017090001C0804100C1814001C0804100C18140C8
:1017190000C1814001C0804100C1814001C08041B8
:1017290001C0804100C1814001C0804100C18140A8
:1017390000C1814001C0804101C0804100C1814098
:1017490000C1814001C0804100C1814001C0804188
:1017590001C0804100C1814000C0C101C30302C270
:10176900C60607C705C5C404CC0C0DCD0FCFCE0ED8
:101779000ACACB0BC90908C8D81819D91BDBDA1A48
:101789001EDEDF1FDD1D1CDC14D4D515D71716D6B8
:10179900D21213D311D1D010F03031F133F3F23228
:1017A90036F6F737F53534F43CFCFD3DFF3F3EFE98
:1017B900FA3A3BFB39F9F83828E8E929EB2B2AEA08
:1017C900EE2E2FEF2DEDEC2CE42425E527E7E62678
:1017D90022E2E323E12120E0A06061A163A3A262E8
:1017E90066A6A767A56564A46CACAD6DAF6F6EAE58
:1017F900AA6A6BAB69A9A86878B8B979BB7B7ABAC8
:10180900BE7E7FBF7DBDBC7CB47475B577B7B67637
:1018190072B2B373B17170B05090915193535292A7
:1018290096565797559594549C5C5D9D5F9F9E5E17
:101839005A9A9B5B99595898884849894B8B8A4A87
:101849004E8E8F4F8D4D4C8C4484854587474686F7
:0818590082424383418180407B
:103FB30052668D00000000000000000000000000B9
:053FC3000000000000F9
:013FF60022A8
:03002300023AC1DD
:103AC100C0E0C083C082C0D075D01830982CE556B4
:103AD10025E9F5EB30D709E55525F904F5FB800615
:103AE100E55525F9F5FBD29174562558F582E43454
:103AF10069F583E599F00558C29830992DE559C3C8
:103B010095575015D290AF59055974562FF582E447
:103B1100346AF583E0F599800FAF578F59EF60084C
:103B2100C2190559D296C290C299D0D0D082D08301
:033B3100D0E032AF
:103EE100C2A9438902758C48758A4875D90475DB66
:103EF1004875DC4875DD4875DE48E4F5E9F5F9C239
:063F0100D9D28CD2DE22B1
:102B58007BFF7A1379F9121D099068AFE07014753C
:102B68002EFF752F147530507BFF7A147912121DC1
:102B7800098012752EFF752F1475305F7BFF7A144C
:102B88007912121D097BFF7A14796E121D09906A59
:102B980078E0FEA3E0FFC3E49FFFE49EFEAB07FAE4
:102BA8003395E0F9F87F007E8C7D0A7C001220E3E3
:102BB8008F318E308D2F8C2E7BFF7A14798F121DDA
:102BC800097BFF7A1479BB9068B0E0F52E121D09D5
:102BD800E4F52A7BFF7A1479DF852A2EE52AFD336E
:102BE80095E0FC74C32DF58274683CF583E0F52FFD
:102BF800AF2AEF3395E0FEEF25E0FFEE33FE74D405
:102C08002FF58274683EF583E0F530A3E0F5317462
:102C1800F42DF58274683CF583E0F532AF2AEF3382
:102C280095E0FE74052FF58274693EF583E0F5336F
:102C3800E52A04F534121D09052AC3E52A6480949F
:102C4800904090906A76E0FEA3E0FF7C007D0A1237
:0F2C580020038E2E8F2F7BFF7A157914121D0902
:012C6700224A
:1022C9007E157F33123747EF4E70037F0122E4906A
:1022D90068AFF07E157F36123747EF4E601B123F0D
:1022E900C98F25E525B431069068AF740AF0E52554
:1022F900B432069068AF7464F07E157F3C1237479C
:10230900EF4E600D123D348F298E288D278C268043
:102319000BE4752980752825F527F526AB29AA2808
:10232900A927A8267F007E8C7D0A7C001220E31253
:102339002175906A78EEF0A3EFF0E47B0AFAF9F8D8
:10234900AF29AE28AD27AC261220E3A804A905AA17
:1023590006AB07E47F307E75FDFC1220E38E558FB6
:10236900567E157F42123747EF4E600A123D349070
:1023790068B0EFF08005E49068B0F07E157F4812F0
:102389003747EF4E6016123D34E47B0AFAF9F8122A
:102399002058906A76EEF0A3EFF0800A906A76747E
:1023A90001F0A374F4F0E4F554F525E525FD339522
:1023B900E0FC74C32DF58274683CF583E4F0E525EF
:1023C900FB3395E0FAEB25E0FFEA33FE74D42FF5F1
:1023D9008274683EF583E4F0A3F074F42DF58274F9
:1023E900683CF583E4F0AF25EF3395E0FE74052FE3
:1023F900F58274693EF583E4F074B12FF58274684F
:102409003EF583E4F0749F2FF58274683EF583747A
:102419000FF0EBAE027803C333CE33CED8F924E103
:10242900F58274153EAF82FE123747EF4E700302F4
:1024390024CA123D34E525FD3395E0FC74C32DF51E
:102449008274683CF583EFF074C32DF58274683C9F
:10245900F583E0606C123D34AD07AC06AF25EF3370
:1024690095E0FEEF25E0FFEE33FE74D42FF582747C
:10247900683EF583ECF0A3EDF0123D34E525FD331C
:1024890095E0FC74F42DF58274683CF583EFF01245
:102499003D34E525FD3395E0FC74052DF58274691D
:1024A9003CF583EFF074B12DF58274683CF583E552
:1024B90054F074F42DF58274683CF583E02554F5E5
:1024C900540525C3E5256480949050030223B4750F
:0424D90054FF7F002D
:0124DD0022DC
:103BA50043AB01C2E8C2EAE4FFEFC454F0F5B1C388
:103BB500EF64809488500575B3D08003E4F5B3E4D1
:103BC500F5B275BCC8F5BDF5BE75BF7875C4FFF512
:103BD500C5F5C675C778F5A3F5A3F5A3F5A3F5A3B4
:103BE500F5A3F5A3F5A30FBF0EBF9068AFE0FF25C2
:103BF500E0F5B475B50C75B66C75A11275AB0275AB
:083C0500C13E75C3FF75C20347
:013C0D002294
:103CD40075B180E4F5B3F5B28545BCE5465403FF00
:103CE40033333354F8FFE54654E04FFFE547C4133C
:103CF40054074FF5BDE54733333354F8FFE548C463
:103D04001354074FF5BEE54833333354F8F5BF85F4
:103D14004AA3854BA3854CA3854DA3854EA3854F0C
:103D2400A38550A38551A3E549540F2450F5B3222C
:102C6800E59B541F6020200B1A7E157F4E12307092
:102C7800E59B541FFF7E007D031231587E157F5857
:102C8800123070E4F59BE5BA30E008E4F5B375B1AD
:102C980080F5B2E5CFF47003022D72752901E4F5D1
:102CA80028E5CFF455297003022D60E528C454F0B7
:102CB800F5B1E5B2547F6420706FE5B3540FF54960
:102CC80085BC45E5BD541FFF131313541FFFE5BD15
:102CD80054E044184FF546E5BDC43354E0FFE5BE63
:102CE800131313541F4FF547E5BEC43354E0FFE5F3
:102CF800BF131313541F4FF54885A34A85A34B856B
:102D0800A34C85A34D85A34E85A34F85A35085A3CA
:102D180051E4F5B2E545547EB5450575B3508003D9
:102D280075B3D0E5492405FF22E5B2549F602320FE
:102D38000B207E157F5B123070AFB27E007D0312D0
:102D48003158AFB37E007D031231587E157F66126D
:102D58003070E4F5B275B3D0E52925E0F5290528EA
:0C2D6800E528C394085003022CA97F004A
:012D7400223C
:103A4700C219E4F558F50BD296F557F559FF7F40A3
:103A5700906916E4F0A3DFFC7F40E4F55AF55C12A9
:103A670022C9123BA5C2ADE4F5C9D2CDD2CCC2C999
:103A7700C2CAF5CDF5CC906A78E0F5CBA3E0F5CADC
:103A870085CBCD85CACCE4F598D29E438740C29FAB
:103A9700C2ACC298C29975B81075B710D2CAD29C79
:103AA700D2AC123EE1C2D9E5E92464F5EB30D70682
:093AB700E5F904F5FB2285F9FB99
:013AC00022E3
:013FF70022A7
:013FF80022A6
:05001E00D29CD2AC22CF
:013FF90022A5
:063E3100AC05AB07AA0678
:103E370090690474FFF0906915F0AF041CEF602DD2
:103E47000BEBAE0270010A14F5828E83E0FF9069D6
:103E570004E06FFF90166193FE906915E06E90691C
:0D3E670004F0EF90176193906915F080CD85
:013E7400222B
:103B340074C32554F582E43468F583E0906A56F042
:103B440074052554F582E43469F583E0906A57F0EE
:103B5400E55425E024D4F582E43468F583E0FCA33D
:103B6400E0FDEC906A58F0A3EDF0E4A3F074F425C2
:103B740054F582E43468F583E0906A5BF07E6A7FF2
:103B8400567D06123E31906904E0906A5CF09069BB
:103B940015E0906A5DF0E4F559755708C296D2991C
:013BA40022FE
:10351F00E55CC394404003E4F55C7416255CF582CA
:10352F00E43469F583E0FF30E16F7416255CF582B2
:10353F00E43469F583EF54FDF0E4906475F0A374FF
:10354F000DF090667AE0906477F0A37419F0A3748D
:10355F0048F0A37479F0E55C131313541FFF9068C0
:10356F00B0E02F90647BF0E55C540725E025E02464
:10357F0080A3F0A37408F0F5F0E55CA4249FF58216
:10358F00E5F03466F58363A20190647E63A2017F48
:0E359F00081225B9055C7F0122055C7F002221
:013FFA0022A4
:100EB1003000469080E8E0700F123C71300D077EE3
:100EC100157F68123070C21B9080E8E0B40E12905A
:100ED10080037408F0300D077E157F71123070C2E7
:100EE1001B9080E8E0B4060F201B0C300D077E1527
:100EF1007F7C123070D21BC200201B03020FB32073
:100F010019071232398F258003E4F525E52560475D
:100F1100300D0C7E157F927C6A7D7EFB122D75E56E
:100F2100E92410F5EB30D708E5F92428F5FB800614
:100F3100E5F92427F5FB906A7E63A201906A566366
:100F4100A201AF251225B9852557E4F559D290C2E2
:100F510091D219C296D29920D9030213F8C2D9E5C8
:100F6100E92410F5EB30D708E5F92428F5FB8006D4
:100F7100E5F92427F5FBE558D3940050030213F853
:100F8100C29185585BE4F55890695663A201906A55
:100F91007E63A201AF5B1225B9AF5B122F80200DDA
:100FA100030213F87E157F977C6A7D7EAB5B122D61
:100FB10075227416255AF582E43469F583E020E040
:100FC10002055AE55AC394404003E4F55A122C68CD
:100FD100EF6069E548640F70639068B0E0FF6547B2
:100FE100705A7416255AF582E43469F583E0FE30AF
:100FF100E04A7416255AF582E43469F583EE54FE0D
:10100100F0754548754679E55A131313541FFEEFE1
:101011002EF547E55A540725E025E02480F548756B
:10102100490875F008E55AA4249FF582E5F0346675
:10103100F5837D4A7F081225B0123CD4300249C2A3
:10104100029068C2E004F070069068C1E004F0D339
:101051009068C2E094B89068C1E0940B402AE4F033
:10106100A3F0F52574162525F582E43469F583E0AE
:1010710030E20E74162525F582E43469F583740394
:10108100F00525E525B440DC20D9030213F8E55726
:101091007003021373E558D39400500302125DC22A
:1010A1009185585B74B12554F582E43468F583E089
:1010B10075F002A485F026F527E4F5587E697F5680
:1010C100906958E02405FD123E31200B0D7E157FFD
:1010D1009C7C697D56AB5B122D75906915E0FF9084
:1010E1006904E04F6010300B030213737E157FA378
:1010F10012307002137374C32554F582E43468F519
:1011010083E0FF906956E06F6010300B03021373A8
:101111007E157FAE12307002137374052554F5826B
:10112100E43469F583E0FF906957E06F6010300B9C
:10113100030213737E157FBD12307002137374F4B2
:101141002554F582E43468F583E075F002A4FF903C
:101151006958E06F7002E5F06010300B0302137301
:101161007E157FCA123070021373749F2554F58265
:10117100E43468F583E4F0F525906958E0FFE5254E
:10118100C39F4003021373749F2527F5827466354C
:1011910026F583E0FF745A2525F582E43469F58349
:1011A100E0FEEF6E6027749F2527F5827466352671
:1011B100F583EEF0E527AE267803CEC313CE13D820
:1011C100F92416F58274693EF5837407F0E527AEBC
:1011D100267803CEC313CE13D8F92416F582746989
:1011E1003EF583E04404F00527E527700205262437
:1011F1009FF58274663526F583E0FF74592525F540
:1012010082E43469F583E0FEEF6E6027749F252741
:10121100F58274663526F583EEF0E527AE26780370
:10122100CEC313CE13D8F92416F58274693EF58323
:101231007407F0E527AE267803CEC313CE13D8F991
:101241002416F58274693EF583E04404F00527E530
:1012510027700205260525052502117A749F25545C
:10126100F582E43468F583E004F0749F2554F58237
:10127100E43468F583E0D3940A5003021373749F36
:101281002554F582E43468F5837405F074B125546E
:10129100F582E43468F583E075F002A485F026F563
:1012A10027E4F52574F42554F582E43468F583E0E8
:1012B100FFE525C39F4003021373749F2527F58221
:1012C10074663526F583E0F46028749F2527F5823E
:1012D10074663526F58374FFF0E527AE267803CED4
:1012E100C313CE13D8F92416F58274693EF58374BD
:1012F10007F0E527AE267803CEC313CE13D8F92421
:1013010016F58274693EF583E04404F00527E5276C
:1013110070020526249FF58274663526F583E06404
:101321007F6028749F2527F58274663526F58374BE
:101331007FF0E527AE267803CEC313CE13D8F92468
:1013410016F58274693EF5837407F0E527AE2678B9
:1013510003CEC313CE13D8F92416F58274693EF572
:1013610083E04404F00527E52770020526052502E0
:1013710012A5906A76E0FEA3E0FF4E6022201A1DBE
:10138100C2D9E025E9F5EB30D708EE25F904F5FBE4
:101391008008906A76E025F9F5FBD21A22C21A0577
:1013A10054E4F557E554C39410504974C32554F5DA
:1013B10082E43468F583E0603E74F42554F582E4F8
:1013C1003468F583E06030C2D9123B34E5E924E8A2
:1013D100F5EB30D708E5F92404F5FB8006E5F9249F
:1013E10003F5FB200B117E157FD87C6A7D567B08A7
:0713F100122D75227554FF57
:0113F80022D2
:033FF3007F00222A
:1035B900020853E493A3F8E493A34003F68001F2CD
:1035C90008DFF48029E493A3F85407240CC8C33313
:1035D900C4540F4420C8834004F456800146F6DFE2
:1035E900E4800B0102040810204080903FADE47E86
:1035F900019360BCA3FF543F30E509541FFEE493D7
:10360900A360010ECF54C025E060A840B8E493A39D
:10361900FAE493A3F8E493A3C8C582C8CAC583CAC8
:10362900F0A3C8C582C8CAC583CADFE9DEE780BE80
:013FC80000F8
:10200300BC000BBE0029EF8DF084FFADF022E4CCC1
:10201300F875F008EF2FFFEE33FEEC33FCEE9DEC8A
:10202300984005FCEE9DFE0FD5F0E9E4CEFD22EDD0
:10203300F8F5F0EE8420D21CFEADF075F008EF2F1A
:10204300FFED33FD4007985006D5F0F222C398FD0B
:052053000FD5F0EA22A8
:10205800E88FF0A4CC8BF0A42CFCE98EF0A42CFC27
:102068008AF0EDA42CFCEA8EF0A4CDA8F08BF0A4A5
:102078002DCC3825F0FDE98FF0A42CCD35F0FCEB04
:102088008EF0A4FEA9F0EB8FF0A4CFC5F02ECD39C9
:0F209800FEE43CFCEAA42DCE35F0FDE43CFC2236
:1020A70075F008758200EF2FFFEE33FECD33CDCCF0
:1020B70033CCC58233C5829BED9AEC99E582984073
:1020C7000CF582EE9BFEED9AFDEC99FC0FD5F0D650
:1020D700E4CEFBE4CDFAE4CCF9A88222B800C1B97A
:1020E7000059BA002DEC8BF084CFCECDFCE5F0CBB8
:1020F700F97818EF2FFFEE33FEED33FDEC33FCEBF1
:1021070033FB10D703994004EB99FB0FD8E5E4F9AB
:10211700FA227818EF2FFFEE33FEED33FDEC33FC98
:10212700C933C910D7059BE99A4007EC9BFCE99A8C
:10213700F90FD8E0E4C9FAE4CCFB2275F010EF2FD1
:10214700FFEE33FEED33FDCC33CCC833C810D707D1
:102157009BEC9AE899400AED9BFDEC9AFCE899F80C
:0E2167000FD5F0DAE4CDFBE4CCFAE4C8F9229F
:0E217500C3E49FFFE49EFEE49DFDE49CFC227B
:10218300EB9FF5F0EA9E42F0E99D42F0E89C45F0B2
:012193002229
:0C219400ECF0A3EDF0A3EEF0A3EFF022BE
:1021A000A8828583F0D083D0821221B71221B71282
:1021B00021B71221B7E473E493A3C583C5F0C583A7
:1021C000C8C582C8F0A3C583C5F0C583C8C582C889
:0121D00022EC
:101CA700E53A242EF8E6053A22782B301702782EEB
:101CB700E475F0011222290221D12010EB7F2ED2E8
:101CC700108018EF540F2490D43440D4FF30140BF5
:101CD700EF24BFB41A0050032461FFE53B600215EF
:101CE7003B053EE53E7002053D30170D782BE47548
:101CF700F001122229EF022217023DEA7403D217DC
:101D07008003E4C217F53A8B2B8A2C892DE4F53B27
:101D1700F53DF53EE53B60077F20121CE280F57537
:101D27003CFFC211C210C212C213C215C216C2189A
:101D3700121CB0FF700D3017057F00121CF3AF3E69
:101D4700AE3D22B4255FC2D5C214121CB0FF24D009
:101D5700B40A00501A75F00A783B30D50508B6FF6B
:101D67000106C6A426F620D5047002D21380D92412
:101D7700CFB41A00EF5004C2E5D214021EF3D211F9
:101D870080C6D21080C0D21280BCD2D580BAD215FC
:101D970080B47F20121CE22012077401B53B00407B
:101DA700F1121CA7FF121CE2021D1BD218D21680CB
:101DB70095121CA7FB121CA7FA121CA7F94A4B7015
:101DC7000679C47A1F7BFF20122EE53B602A7E002E
:101DD7008E827583001221EA60060EEE653C70F074
:101DE700C2D5EBC0E0EAC0E0E9C0E0EE121F3AD08E
:101DF700E0F9D0E0FAD0E0FB1221D1FF60AAEBC0F6
:101E0700E0EAC0E0E9C0E0121CE2D0E02401F9D02A
:101E1700E03400FAD0E0FBE53C0460DCD53CD98037
:101E2700877BFF7A1F7936D212809C7910800279DE
:101E370008C216C2188008D2D5790A8004790AC266
:101E4700D5E53C047002F53CE4FAFDFEFF121CA741
:101E5700FC7B08201113121CA7FD7B1030100A12FF
:101E67001CA7FE121CA7FF7B20EC3382D592D5500E
:101E770013C3E43010069FFFE49EFEE42011039D88
:101E8700FDE49CFCE4CBF8C211EC700CCFCECDCCBA
:101E9700E824F8F870F38017C3EF33FFEE33FEED55
:101EA70033FDEC33FCEB33FB994002FB0FD8E9EB36
:101EB700301105F8D0E0C448B211C0E00AEC4D4E2D
:101EC7004F78207B0070C2EAB53C0040BCC0E012EE
:101ED7001F3CD0F0D0E0201104C4C0E0C4B211C050
:101EE700F0121CCBD0F0D5F0EB021D1B1222881D7F
:101EF700B8531E32581D894C1D85421E364F1E3E53
:0F1F0700441E3E491D9E431E44551E28461E285B
:101F1600451E28471FE4501D8D2D1D912E1DB42BE7
:101F26001D95231DB2201FCD2A1D4D4800001DAC56
:101F36003F3F3F00790AA2D5201314301509B91086
:101F4600020404B9080104A2D52016025001042097
:101F560012689212B53B005034C0E07F203013194E
:101F66007F30A21272167215500F121F93C212C240
:101F760016C215C2187F30800F301503E9C0E01273
:101F86001CE2301503D0E0F9D0E0B53BCC30151794
:101F96007F30B9100C121CE27F583014077F78800E
:101FA60003B90803121CE23012057F2D021CE27FE2
:101FB600202018F87F2B2016F322921280CF286E4D
:101FC600756C6C2900D211121CA73011F8C2117859
:101FD6003B30D50108F6021D4D2D50434958121CC1
:101FE600A72403B405004001E4901FDF93121CD31D
:0D1FF600743A121CD3D213753B04021E3244
:1026C7008B2A8A2B892CE4F536F535F534F533F565
:1026D70031F532E52E452F452D6012EBC0E0EAC0FB
:1026E700E0E9C0E0AB2DAA2EA92F122239AB2A05AB
:1026F7002CE52CAA2B7002052B14F91221D1F537E2
:10270700C394094007E537D3940D40E1E5376420CA
:1027170060DBE537B42D054332038016E537B42B6C
:1027270005433201800C74FF252CF52C74FF352BE3
:10273700F52BE53060046410703FAB2AAA2BA92C57
:102747001221D164306009E530702E75300A802976
:102757009000011221EAFF64786004EFB458134334
:1027670032017530107402252CF52CE4352BF52B2E
:102777008007E5307003753008AB2A052CE52CAAD5
:102787002B7002052B14F91221D1F537C394614040
:102797000AE537D3947A50035337DF74D02537F5DA
:1027A70037C3940A400CE5379411406D74F9253707
:1027B700F537E537D39530506043320185363B8591
:1027C700353A853439853338AF307E00E4FCFDABCC
:1027D70036AA35A934A833122058C8ECC8C9EDC9A0
:1027E700CAEECACBEFCBE4FCFDFEEB2537F536EEA0
:1027F7003AF535ED39F534EC38F533AF36AE35AD5E
:1028070034FCAB3BAA3AA939A838D3122183500329
:10281700022780433204022780E53220E003E48068
:102827002DE52E452F452D601EAB2AE52C24FFF9FB
:10283700E52B34FFFAEBC0E0EAC0E0E9C0E0AB2DDE
:10284700AA2EA92F122239E53230E20774FFFFFEC4
:10285700FDFC22E532AF36AE35AD34AC3330E103A3
:0428670002217522B3
:1021D100BB010689828A83E0225002E722BBFE020C
:0921E100E32289828A83E493223F
:1021EA00BB010CE58229F582E5833AF583E02250AA
:1021FA0006E92582F8E622BBFE06E92582F8E222F4
:0D220A00E58229F582E5833AF583E493220D
:10221700BB010689828A83F0225002F722BBFE01A6
:02222700F322A0
:10222900FAE6FB0808E6F925F0F618E6CA3AF622B6
:10223900BB011A89828A83D0F0D0E0F8D0E0F9D0C6
:10224900E0FAD0E0FBE8C0E0C0F00222B75016E99E
:10225900F8D083D082D0E0F9D0E0FAD0E0FBC08298
:10226900C0830222AEBBFE16E9F8D083D082D0E04B
:0F227900F9D0E0FAD0E0FBC082C0830222C0227D
:10228800D083D082F8E4937012740193700DA3A3E5
:1022980093F8740193F5828883E4737402936860F9
:0622A800EFA3A3A380DFF9
:0922AE00EBF608EAF608E9F62255
:0922B700EBF0A3EAF0A3E9F02228
:0922C000EBF208EAF208E9F2224F
:00000001FF
